:100000003FC058C157C056C055C054C053C052C05D
:1000100051C052C24FC096C24DC04CC04BC04AC026
:1000200049C048C047C0FDCB3CCCFDCB38CC60CCF0
:100030005FCC5ECC5DCC5CCC5BCC5ACC59CC58CC84
:1000400057CC56CC55CC54CC53CC52CC51CC50CCB4
:100050004FCC4ECC39CC4CCC2ACC0ACC3DCCF0CBBE
:100060002CCC46CC45CC44CC06CCDFCB3BCC40CCD6
:100070003ECC3ECC0DCCE9CB3BCCF4CB39CC0CCC3C
:1000800011241FBECFE5D4E0DEBFCDBF11E0A0E656
:10009000B0E0EAE0FFE102C005900D92A633B1079F
:1000A000D9F711E0A6E3B1E001C01D92AE3BB10764
:1000B000E1F72FCCA5CF089580916A00882381F0C5
:1000C00010926A0080916B0097E087FF02C0979AB8
:1000D00001C097989698969A880F915097FFF5CF00
:1000E00008950895E82FFF27EF70F070E053FF4F59
:1000F000808199270895E82FFF27EF70F070E05274
:10010000FF4F808199270895E82FFF27E370F07053
:10011000E051FF4F80819927089597E087FF02C043
:10012000959A01C095989798979A880F915097FF44
:10013000F5CF08951F93CF9380919A018F5F80939D
:100140009A0180919A01833350F010929A0190E0C5
:1001500080917801882309F491E09093780180914F
:10016000850199272091390102C0880F991F2A958E
:10017000E2F787FF06C080917801882311F4C82F29
:1001800007C080913901E82FFF27E05AFE4FC08158
:100190008C2FB1DF182F8C2F82958F70ACDFC82F7A
:1001A00080913901843028F080913901ADDFC82376
:1001B00004C080913901A8DF18237EDF8091680098
:1001C000882379F0812FA9DF8C2FA7DF8091390157
:1001D0008F5F8093390180913901883010F010923F
:1001E0003901CF911F9108958091B90187FD05C014
:1001F0008091B9018F5F8093B9019FE0C498C59841
:10020000C59A915097FFFACFB3993DC090E0809185
:100210003801891711F4C49801C0C49AC598C59AC9
:100220009F5F9031A0F3000000000000B3992DC043
:1002300080913601882399F0909176018091380160
:10024000981769F480913801873021F08091380146
:100250008630D9F48091B9018333B8F009C081E0C8
:10026000809336011092B901809138018093760114
:1002700080913801E82FFF27E054FF4F80818F5F86
:100280008093370102C010923601809138018F5F50
:100290008093380180913801803110F0109238013C
:1002A0000895089580913701882311F01092370145
:1002B000992708951F920F920FB60F9211248F93D2
:1002C0009F939091A201992379F48091A2018F5F6D
:1002D0008093A2019093B801109287011092860139
:1002E00090937501909371019F918F910F900FBE24
:1002F0000F901F901895809175018F5F8093750105
:10030000809175018E3008F061C080916801282FBE
:10031000332727FD30958091A501992787FD90957A
:10032000281B390B37FF03C0309521953F4F2230F2
:1003300031052CF4809171018F5F80937101809160
:100340004D01282F332727FD309580918101992772
:1003500087FD9095281B390B37FF03C030952195F9
:100360003F4F223031052CF4809171018F5F8093D3
:10037000710130E0909168018091A50189170CF41A
:1003800031E020E090914D018091810189170CF4BA
:1003900021E0321729F4809171018F5F8093710100
:1003A0008091860190918701880F991F9093870112
:1003B000809386018091860190918701231708F42C
:1003C000816090938701809386011CC080917501A4
:1003D0008F30C0F080917101882391F48091860163
:1003E00090918701892F992782958F7080FF08C08F
:1003F000809186019091870190937401809373019D
:100400001092A201109281018091810180934D018F
:1004100080914D018093A5018091A5018093680191
:1004200008958C3038F4E82FFF27EC50FF4F80817F
:10043000992708958AE190E0089508951F93809187
:10044000A201882369F18091B8018E3070F0829901
:1004500006C0809181018F5F8093810113C08091DC
:100460004D018F5F80934D010DC0829906C0809130
:10047000A5018F5F8093A50105C0809168018F5F02
:10048000809368018091B801182F8F5F8093B80125
:1004900080917501C6DF811718F41092B8012BDF27
:1004A0001F9108958091B001882321F043DE9CDEE6
:1004B0001092B001089508951F920F920FB60F92F7
:1004C00011242F933F934F935F936F937F938F9359
:1004D0009F93AF93BF93EF93FF93B0DF80915F0142
:1004E0008E3F28F480915F018F5F80935F01809140
:1004F0005F018034B1F410925F018091B0018F5F91
:100500008093B0018091410190914201C29748F4DB
:100510008091410190914201019690934201809314
:100520004101FF91EF91BF91AF919F918F917F9189
:100530006F915F914F913F912F910F900FBE0F9050
:100540001F9018951F920F920FB60F9211248F9340
:100550009F93EF93FF9380914701803160F48091E6
:100560004701E82FFF27E25BFE4F9CB190838F5F2E
:100570008093470101C08CB1FF91EF919F918F91C2
:100580000F900FBE0F901F9018958F9A8D9A8E9A8C
:100590008F9ABD9ABC9ABB98C39AB89A8B9A8C9A38
:1005A000A59AA49AAD9AAC9AA098A198A298A3985B
:1005B00017B885E886B991E093BF89B7892B89BFC1
:1005C000B99ABA9A81EA8FBD9EBD80E780935E0199
:1005D00080E790E09BBD8ABD88EC8093720188EC37
:1005E00090E099BD88BD8A98C29A83E085BF8BB799
:1005F00080648BBF8898899A89E189B988E98AB92A
:1006000078940895CF93DF93EC01CC0FDD1FCC0FCE
:10061000DD1FC80FD91F1C161D0644F443DF80E000
:100620008A95F1F721971C161D06C4F3DF91CF912F
:100630000895CF93C82F8A3011F48DE0FADF5D99C9
:1006400003C030DF5D9BFDCFCCB980E090E0CF915F
:100650000895CF93DF93EC018881882329F0899155
:10066000E8DF88818823D9F7DF91CF910895FF9241
:100670000F931F93F82E82958F7000E011E0F80120
:10068000E80FF11D8081D5DFEF2DFF27EF70F070AF
:10069000E00FF11F8081CDDF1F910F91FF90089532
:1006A000EF92FF920F931F93CF93DF9380919C0162
:1006B00090919D01A0919E01B0919F012AE030E0B0
:1006C00048EA51E0BC01CD0121DB7C01E8EAF1E020
:1006D00001900020E9F73197E85AF1401E2F90E091
:1006E000292F3327E901C05ADE4F8A8184708A831B
:1006F000F901E758FE4F092F0F5F163020F480E311
:1007000080831F5F09C0D7018D917D018083805355
:10071000E9DC9A81982B9A83902F063008F3DF91B9
:10072000CF911F910F91FF90EF900895EF92FF925C
:100730000F931F93CF93DF93162F4AE050E068EAA0
:1007400071E00ADB7C01E8EAF1E001900020E9F7C2
:100750003197E85AF1400E2FC12FDD27C05ADE4FE6
:1007600013E0888184708883043010F40F5F08C020
:10077000F70181917F018053B5DC9881982B988394
:100780001150219617FFEDCFDF91CF911F910F915F
:10079000FF90EF900895EF92FF920F931F93CF93E6
:1007A000DF93809144014AE050E068EA71E09927C4
:1007B00087FD9095D1DA7C01E8EAF1E00190002014
:1007C000E9F73197E85AF1401E2FC0E6D1E001E089
:1007D000888184708883123028F488818B6B8883A9
:1007E0001F5F08C0F70181917F0180537BDC9881F6
:1007F000982B98830150219607FFEACFDF91CF9184
:100800001F910F91FF90EF90089587B980E08A952E
:10081000F1F7369A369B03C045DE3699FDCF80E06E
:100820008A95F1F7369A369B03C03CDE3699FDCFA8
:1008300084B195B10895982F30E027E0E7E6F1E024
:1008400097FD3F5F80818B7F8083332319F0808108
:1008500084608083990F2150319727FFF1CF08954D
:100860000F931F93CF93DF9383E4CFDF9695879504
:1008700096958795082F1127802FDDDF80E2D9DE3E
:100880004AE050E068EA71E0C80166DAEC01E8EAA3
:10089000F1E001900020E9F73197E85AF1400E2F7E
:1008A00013E0043020F480E3C4DE0F5F02C08991BE
:1008B000C0DE115017FFF5CFDF91CF911F910F913F
:1008C0000895E19B03C00000E199FDCF9FBB8EBB63
:1008D0006DBBF894E29AE19A78940895EF92FF92B2
:1008E0001F93CF93DF93EC017B01442349F0142F36
:1008F000CE012196F70161917F01E3DF1150C1F72D
:10090000DF91CF911F91FF90EF900895982F823142
:10091000A8F48091BA01843088F01092BA01892F2E
:100920009927880F991F880F991F42E066EA71E0A6
:1009300080569E4FD3DF80E191E08BDE08950895CD
:10094000E19B03C00000E199FDCF9FBB8EBBE09A05
:100950008DB399270895EF92FF921F93CF93DF9362
:10096000EC017B01442349F0142FCE012196E8DFEE
:10097000F70181937F011150C1F7DF91CF911F9152
:10098000FF90EF900895DF92EF92FF920F931F93E5
:10099000CF93DF93DD24C0EAD1E0EE24FF2404E40A
:1009A00010E042E063EA71E0CE01D5DF809173018F
:1009B0009091740197702091A3013091A4012817A0
:1009C000390709F52091A6013091A70180917301A3
:1009D000909174012817390719F48BE08D1598F45C
:1009E000ADE0AD1558F08091730190917401909332
:1009F000A7018093A601C701019611C0D801ED910E
:100A0000FC9109950AC0D3940894E11CF11C0E5F77
:100A10001F4F2496B1E1BD1520F680E090E0DF91F4
:100A2000CF911F910F91FF90EF90DF900895982F35
:100A300026E030E040E050E067E090FF02C0949A8A
:100A400001C09498822F8A95F1F7939A822F8A9504
:100A5000F1F793989695615067FFEFCF08950F9344
:100A60001F9380919C0190919D01A0919E01B09156
:100A70009F018C0180919C0190919D01A0919E010C
:100A8000B0919F01BC01CD0122E330E040E050E095
:100A9000CAD9CA01B90122E330E040E050E084D96C
:100AA000DC01CB01081B190B88EE97E6801B910B2C
:100AB0009093990180939801809198019091990168
:100AC00065E070E09CD98B01F894C09A862FAFDF67
:100AD000812F9927ACDF80918301E82FFF27EC5EFF
:100AE000FE4F80818093820180918401882329F0C8
:100AF000809182018160809382018091820197DFE1
:100B0000C098949878941F910F910895AD9AAC9ADB
:100B10008DE0982F9A95F1F7AC988A95F1F7AD98FA
:100B20000895AC98AD9A8DE08A95F1F7AC9A089546
:100B30008DE0982F9A95F1F7AD9A8A95F1F7AD98D7
:100B400008951F93CF93C82F17E0C7FF02C0AC9A38
:100B500001C0AC98EDDFCC0F115017FFF6CFE8DFE6
:100B6000CF911F910895EF92FF920F931F93CF9310
:100B7000C1E080919C0190919D01A0919E01B09156
:100B80009F0189579D45A240B04008F0C2E0809186
:100B90009C0190919D01A0919E01B0919F01815C6B
:100BA000964BA640B04008F0CCE080919C0190911B
:100BB0009D01A0919E01B0919F018C549E46AF4F24
:100BC000BF4FBC01CD0122E330E040E050E02BD923
:100BD0007901002711279ADF80ECB3DFBB27A12F13
:100BE000902F8F2DAEDF8E2DACDF80913A018823C0
:100BF00011F089E801C088E8A4DF8C2FA2DF91DF23
:100C0000CF911F910F91FF90EF9008950F931F9335
:100C1000CF9346DD87E191E01CDD83E4F6DDC0E0A3
:100C200009E711E0F80181918F0103DDC23011F471
:100C30008EE2FFDCCF5FC630A8F312DE11DE10DEDD
:100C4000CF911F910F9108950ADF8DDFDFDF0895A7
:100C5000CF93C0E081E4D9DD9695879596958795E9
:100C600090914801292F3327281B310937FF03C0F2
:100C7000309521953F4F2A3031053CF0891710F40B
:100C8000CDE001C0CEE0809348018C2F9927CF9111
:100C9000089580E4BADD9695879596958795282FD7
:100CA0002095809149019927821B910997FF03C0E4
:100CB000909581959F4F03978CF020934901822F47
:100CC00063E091D890E7981B903308F490E39093F9
:100CD0005E0180915E0199279BBD8ABD08950895AC
:100CE0008091B4008823C1F182E48FDD96958795C9
:100CF00096958795982F909580914A01891721F0B4
:100D000090934C0190934A019091BB0180914C01CA
:100D1000891720F080914C01882381F410924001C2
:100D200010923F0110924201109241018091840182
:100D3000882391F01092840192DE08958091410100
:100D400090914201C29740F080918401882321F460
:100D500081E08093840183DE08950895982F809127
:100D60006900882309F445C020913B0130913C0182
:100D7000290F311D30933C0120933B018091A1014B
:100D80008F5F8093A1018A30A0F1C9016AE070E011
:100D900036D870933C0160933B016C3E710570F056
:100DA00080916B00823050F080916B008150809375
:100DB0006B0080916A008F5F80936A0080913B0195
:100DC00090913C01823D910570F480916B008F3FC2
:100DD00051F080916B008F5F80936B0080916A006F
:100DE0008F5F80936A0010923C0110923B01109239
:100DF000A10108950895809143019927009719F062
:100E0000019749F1089520919C0130919D014091F5
:100E10009E0150919F018091B0009091B100A091EE
:100E2000B200B091B300281739074A075B0778F47E
:100E30002091B60080919C0190919D01A0919E010E
:100E4000B0919F01820F911DA11DB11D27C081E0AE
:100E500080934301089520919C0130919D01409120
:100E60009E0150919F018091AC009091AD00A091A6
:100E7000AE00B091AF0082179307A407B507B8F48E
:100E80002091B60080919C0190919D01A0919E01BE
:100E9000B0919F01821B9109A109B10980939C0126
:100EA00090939D01A0939E01B0939F01089510928D
:100EB0004301089508959FDFC7DE089580914B0197
:100EC00099270097B1F0019741F58091B5008F5FA8
:100ED0008093B5008091B500883010F01092B50075
:100EE0008091B500E82FFF27E954FF4F8081809360
:100EF000B6008AED8093600181ED8093610183EDFE
:100F00008093620183E7809363018091B60064E07F
:100F100099270CDC81E080934B010895089580911E
:100F20008301EBE1F1E0E80FF11D80818093610125
:100F3000089580914B018830D1F41092400188EDE2
:100F40009BE0ADE0B0E08093B0009093B100A0933F
:100F5000B200B093B30088EC9FEAA0E0B0E08093C9
:100F6000AC009093AD00A093AE00B093AF00109290
:100F70003F0110924B0183E780936001109285013D
:100F8000CEDF62DE08959B01AC018091B0009091AC
:100F9000B100A091B200B091B30082179307A407EB
:100FA000B50748F18091AC009091AD00A091AE00E2
:100FB000B091AF00281739074A075B07E0F0CA0174
:100FC000B90125E030E040E050E02DD7DA01C90159
:100FD00062E0880F991FAA1FBB1F6A95D1F7820F85
:100FE000931FA41FB51F80939C0190939D01A09314
:100FF0009E01B0939F019DDF089590914B0199232D
:1010000069F4809183018F5F8093830180918301D4
:10101000833010F09093830182DF21DD08950895DD
:10102000882339F0109265018BEB8093660189E487
:1010300006C08BEB8093650183E580936601809306
:1010400067010895089580914B019927009759F001
:101050000297E9F490E080913A01882309F491E045
:1010600090933A0180DD8BE9809360018BE7809358
:10107000610188E28093620189E4809363011092A8
:10108000640180913A01CCDF82E080934B010895A6
:10109000089580914B019927009781F0039711F5EE
:1010A00090E080916900882309F491E090936900B1
:1010B0008FEF80936B0081E080936A0089EB8093CF
:1010C00060018BE78093610183E78093620188EF81
:1010D000809363011092640180916900A1DF83E035
:1010E00080934B01089508958FEF80936C01809356
:1010F0006B0180936A018093690180914401992773
:1011000087FD909544E069E671E0880F991F880F8C
:10111000991FE4DB089580914B0199278430910554
:1011200049F0853091051CF4892B21F0089506972C
:10113000B9F00895F4DE80E28093850183E5809321
:10114000600180E88093620185E0E3E6F1E01192BE
:101150008A95E9F71092770184E080934B01089516
:10116000C3DF8FEF8093850180ED97E04BDA80EC51
:101170008093850108950895FF920F931F93F82E91
:101180008091850186958093850180917701E82F74
:10119000FF27E05AFE4F828184708283809177011D
:1011A000082F1127005A1E4F8F2D9CD7F8019281CE
:1011B000982B928380917701E82FFF27EF54FE4F01
:1011C00090E3F90EF0828F5F809377018091770131
:1011D000E82FFF27EF54FE4F108280917701863071
:1011E00068F04AE050E060E070E081EB91E08ED47E
:1011F000DC01CB01BC01CD01C6DE08C080917701C6
:10120000E82FFF27E05AFE4F80E882831F910F915D
:10121000FF90089580E0B0DF089581E0ADDF08958C
:1012200082E0AADF089583E0A7DF089584E0A4DFC9
:10123000089585E0A1DF089586E09EDF089587E0A8
:101240009BDF089588E098DF089589E095DF089591
:10125000CF93FC01C62F80914B01282F33272115F6
:10126000310589F025303105C1F444E06CE971E0C5
:10127000CF0134DB10928501C093600180ED97E0CF
:10128000C1D957DE0AC080E8809385016093600170
:101290001092610185E080934B01CF91089569E739
:1012A0008CEF91E0D5DF089561E988EF91E0D0DF20
:1012B000089580914401992787FD909544E069E65F
:1012C00071E0880F991F880F991F45DB20916C01F1
:1012D000822F992783709070039751F446E050E075
:1012E00060E470E082E691E00AD481E090E0089545
:1012F00023702093830183E0A9E6B1E0ECE9F1E0FB
:101300000D9001928A95E1F79FDC80E090E00895CE
:101310000895CF9380914401282F332727FD3095DE
:1013200080913D01A82FBB27A7FDB095FD01E25E8E
:10133000FE4FE0818E2F9927281739076CF0809196
:101340004401282F332727FD3095AE5DBE4F8C9189
:1013500099278217930714F4E0934401C091440144
:10136000809144018F5F8093440180914401282F34
:10137000332727FD309580913D01A82FBB27A7FD7E
:10138000B095FD01EE5DFE4F80819927821793078E
:101390002CF4A25EBE4F8C91809344018ADF882397
:1013A00039F45EDA5DDA5CDA5BDA5ADA59DA0AC005
:1013B0002C2F332780914401992787FD909528177A
:1013C000390771F6E8D9CF91089580914B018823B0
:1013D00029F481E0809343010EDD36DC80914B01DE
:1013E000863021F080914B01873091F48091440147
:1013F0008150809344018091440187FF03C083E6BC
:1014000080934401C8D980914B01873009F451DFA2
:1014100080914B018930A9F480919B01882389F444
:1014200080913D01815080933D0187FF03C083E09F
:1014300080933D0180913D0164E0992787FD90955F
:1014400075D90895089580914B01882321F48093E4
:101450004301D1DCF9DB80914B01863021F0809192
:101460004B01873089F4809144018F5F8093440160
:1014700080914401843614F0109244018CD98091FB
:101480004B01873009F415DF80914B018930A1F4BD
:1014900090919B01992381F480913D018F5F80930E
:1014A0003D01843014F090933D0180913D0164E052
:1014B000992787FD90953AD90895089580919C01C8
:1014C00090919D01A0919E01B0919F01809369012F
:1014D00090936A01A0936B01B0936C01809183019A
:1014E0008C6F80936C0180914401992787FD9095C2
:1014F00044E069E671E0880F991F880F991FEED9C3
:10150000089580914B019927009751F0069779F43F
:10151000D5DF1092850180ED97E074D80ADD08953B
:1015200080EC8093850137D986E080934B01089544
:10153000089580914B01882329F487E080934B0123
:101540002AD9B7DE0895089580914B01883041F47F
:1015500090E080914001882309F491E0909340014C
:1015600080914B01882309F0A4C088E080934B014F
:101570008BE380936001D3DC44E060EB70E08CEFA0
:1015800091E0E9D944E06CEA70E088EF91E0E3D9BA
:101590002091B0003091B1004091B2005091B30061
:1015A0008091AC009091AD00A091AE00B091AF00E1
:1015B000281739074A075B0760F444E060EB70E0E6
:1015C00088EF91E0C8D944E06CEA70E08CEF91E0DC
:1015D000C2D98091B0009091B100A091B200B091B9
:1015E000B300B7FF0CC088ED9BE0ADE0B0E08093A6
:1015F000B0009093B100A093B200B093B30080917B
:10160000AC009091AD00A091AE00B091AF00B7FFDB
:101610000CC088EC9FEAA0E0B0E08093AC0090930F
:10162000AD00A093AE00B093AF0020919C0130912B
:101630009D0140919E0150919F018091B000909139
:10164000B100A091B200B091B30082179307A40734
:10165000B507C8F020919C0130919D0140919E01F9
:1016600050919F018091AC009091AD00A091AE008F
:10167000B091AF00281739074A075B0720F0809127
:101680003E01882399F08091AC009091AD00A0912B
:10169000AE00B091AF0080939C0190939D01A09308
:1016A0009E01B0939F0110923E01CEDA81E08093BB
:1016B000400108950895CF9380914B01893091F4B2
:1016C00080919B01882349F090E080913F0188231D
:1016D00009F491E090933F0105C081E080933F01C0
:1016E00080939B01C0914B01CC23C1F489E080938E
:1016F0004B0189ED809360018BE78093610189E460
:101700008093620181EC8093630180913D0164E0EC
:10171000992787FD90950AD8C0939B01CF91089592
:101720001F93CF93DF93CDB7DEB724970FB6F8940E
:10173000DEBF0FBECDBF80914B01882329F0809181
:101740004B01883009F0DBC0909147018091460140
:10175000981709F4D4C080914601E82FFF27E25B77
:10176000FE4F8F5F8093460110811A3031F08091D7
:10177000BF00882311F0812F5CD780914701803111
:1017800048F010924501109247011092460186E2FE
:1017900091E0B4C0812F992768D3892B51F08091B3
:1017A0004501E82FFF27E857FE4F10838F5F809396
:1017B00045011D3009F0A3C080914501E82FFF27A6
:1017C000E857FE4F10821092450180914B018830FE
:1017D00019F410924E01ADDB4AE050E060E070E099
:1017E00088E891E093D1DC01CB0189839A83AB83B4
:1017F000BC83298110E080914E018A3009F411E008
:10180000E12FFF27E25BFE4F80819927AA27BB27A4
:10181000FC01BB97ED32F10508F06AC0ED5EFF4FA9
:10182000099411DE65C0D1DD63C02370209383016C
:1018300080918301833011F41092830170DB26C004
:10184000217020933A018FD953C027702093B5009F
:101850008091B500E82FFF27E954FF4F80818093E6
:10186000B60046C020936B0081E080936A0040C0C0
:101870002093BF003DC0223021F481E08093B4006A
:1018800037C02170209384011092B400E8D830C092
:1018900021702093A0012CC0822F38D829C0B6D93E
:1018A00027C0DED7DDD7DCD7DBD7DAD721C02223AC
:1018B000F9F081E0809368001BC044E0BE016F5FD7
:1018C0007F4F8CEF91E006C044E0BE016F5F7F4F19
:1018D00088EF91E003D80CC069817A818B819C816B
:1018E00052DB06C080913E018F5F80933E012CDE6B
:1018F00010924701109246018DE291E0AAD62496FB
:101900000FB6F894DEBF0FBECDBFDF91CF911F9110
:101910000895CFE5D4E0DEBFCDBF37D611E01093F8
:1019200084011092830188E690EAA1E0B0E0809300
:101930009C0190939D01A0939E01B0939F01B9DCFF
:10194000F8DA88EE93E05ED61093A00181D9AAD58B
:10195000E7DEA8D4182F8091730190917401892B30
:1019600009F441C0C091A001CC2319F00CD8182F64
:1019700036C080E391E06DD680917301909174013F
:10198000892F992774D680917301909174016FD635
:101990008DE291E05ED68091730190917401977011
:1019A00090937401809373012091730130917401BD
:1019B0008091A6019091A7012817390731F48091F1
:1019C000BA018F5F8093BA010AC0C093BA018091B7
:1019D0007301909174019093A7018093A6011092D6
:1019E00074011092730155D9112311F431D9182FB4
:1019F00011501F3F89F0E12FFF27EF70F0708091A9
:101A00004B01843009F4E061EE0FFF1FE459FF4FF2
:101A10000190F081E02D09958091400181114BDA10
:101A200080913F01811175DC83E4EFD6969587950F
:101A3000969587958093BB018091BB01FCD650D9C8
:101A40008091BB018BD983CF80914C01843658F0B3
:101A500080914C01865F80934C0180914C018A30CB
:101A600088F48FEF07C080914C01853130F0809170
:101A70004C018B5F80934C01089580914C018F5FE6
:101A800080934C010895089580914C01843620F094
:101A900080914C018A5007C080914C018A3130F00E
:101AA00080914C01855080934C01089580914C01A8
:101AB000882329F080914C01815080934C01089536
:101AC000089580915E01813348F080915E01282F56
:101AD0003327815080935E013BBD2ABD0895089550
:101AE00080915E01803748F480915E01282F332772
:101AF0008F5F80935E013BBD2ABD08950895DC0190
:101B000001C06D9341505040E0F70895A0E0B0E06F
:101B1000EBE8FDE0C5C18C012B01EA01EE24611563
:101B2000710519F0FB0180839183209749F0CE0164
:101B30000297839728F060E070E080E090E0E2C0D8
:101B4000F801F1908F018F2D992799D1892BC1F739
:101B5000FDE2FF1619F441E0E42E03C0FBE2FF169C
:101B600019F4F801F1908F01209719F0C031D105D7
:101B700091F4F0E3FF1679F4F8018081883711F0D1
:101B8000883549F4F801F1800E5F1F4FC0E1D0E0C5
:101B9000F2E0EF2A0AC0209741F480E3F81619F426
:101BA000C8E0D0E002C0CAE0D0E0C830D105E9F01A
:101BB000C930D10524F4C230D105E9F022C0CA30C1
:101BC000D10521F0C031D10551F01BC03CECA32E52
:101BD0003CECB32E3CECC32E3CE0D32E1EC0A12C1B
:101BE000B12CC12C28E0D22E18C0A12CB12CC12CB4
:101BF00090E1D92E12C0A12CB12CC12C80E4D82E9A
:101C00000CC09E01442737FD4095542F60E070E0E2
:101C100080E090E808D159016A0120E030E040E01E
:101C200050E060E03E01882477FC8094982C8F2D52
:101C300080538A3010F4F82E0DC08F2D81548A31D4
:101C400018F4E9ECFE0E06C08F2D81568A3140F55E
:101C5000F9EAFF0E8F2D99278C179D070CF567FD6C
:101C60001BC0A216B306C406D50698F0CA01B90176
:101C7000A401930199D09B01AC012F0D311D411D91
:101C8000511D213080E0380780E0480780E8580780
:101C900010F06FEF01C061E0F801F1908F01C7CF44
:101CA0004114510461F0662319F00150104004C042
:101CB000E1FE05C002501040F201008311838E2D19
:101CC000992767FF07C080FF11C020E030E040E0A7
:101CD00050E810C080FF08C0509540953095219580
:101CE0003F4F4F4F5F4F0CC057FF0AC02FEF3FEFE2
:101CF0004FEF5FE782E290E09093BD018093BC01DB
:101D0000CA01B901E0E1CDB7DEB7E6C0F52FE42F97
:101D1000CF93FF93EF932230D4F02532C4F4C22F37
:101D20002C2F332744275527FF93EF937CD0EF9137
:101D3000FF91605D6A330CF0695D6193622F732FD0
:101D4000842F952F605070408040904049F710825A
:101D50008F919F91CF9118C0E62FF72F2E2F3F2FF5
:101D6000423074F0453264F4642F772748D0805DA8
:101D70008A330CF0895D8193862F972F0097A1F706
:101D8000932F822F108200C0DC01FC010190002003
:101D9000E9F73297AE17BF0730F47C91608170830A
:101DA00031976D93F7CF0895629FD001739FF00133
:101DB000829FE00DF11D649FE00DF11D929FF00DDB
:101DC000839FF00D749FF00D659FF00D9927729F12
:101DD000B00DE11DF91F639FB00DE11DF91FBD019D
:101DE000CF0111240895991B79E004C0991F96171B
:101DF00008F0961B881F7A95C9F780950895AA1B4D
:101E0000BB1B51E107C0AA1FBB1FA617B70710F0E5
:101E1000A61BB70B881F991F5A95A9F78095909517
:101E2000BC01CD010895A1E21A2EAA1BBB1BFD0126
:101E30000DC0AA1FBB1FEE1FFF1FA217B307E407A9
:101E4000F50720F0A21BB30BE40BF50B661F771F01
:101E5000881F991F1A9469F76095709580959095E1
:101E60009B01AC01BD01CF010895992329F4803372
:101E70001CF08A330CF40895992788270895992334
:101E8000D9F78032D9F38A30C9F38C30B9F38D3069
:101E9000A9F3893099F38B3079F708952F923F9207
:101EA0004F925F926F927F928F929F92AF92BF926A
:101EB000CF92DF92EF92FF920F931F93CF93DF9316
:101EC000CDB7DEB7CA1BDB0B0FB6F894DEBF0FBE73
:101ED000CDBF09942A88398848885F846E847D84C0
:101EE0008C849B84AA84B984C884DF80EE80FD80C2
:101EF0000C811B81AA81B981CE0FD11D0FB6F89438
:0A1F0000DEBF0FBECDBFED01089556
:101F0A00240D440D610D700D010101FFFD075E07EF
:101F1A00230849084F09810A5409A40A990A5B0B44
:101F2A008B089907230AE5095B005B000A090D097A
:101F3A0010091309160919091C091F09220925097B
:101F4A008B0899075B005B005B005B00C8AF000071
:101F5A00D80B0D0001010A050A0F14191E3264017B
:101F6A000000020306090D0C08040501000A0B070C
:101F7A00BB28E3EA78DADB2AFBFA7BD993E9D35365
:101F8A0065676D6F75777D7FE5E7EDEFF5F7FDFF27
:101F9A00BFDFFBFE1A1A191A1A1A191A1A1A191A6B
:101FAA003031323334353637383941424344454685
:101FBA000A4F4B00E6E4E20A462000C8C1C90119EB
:101FCA00324B18314A630A4572720A3E000A3E00D1
:061FDA005243353A0000FD
:00000001FF
